:100000000EC0189518951895189518951895189567
:1000100018951895189518951895189518958FE5B1
:100020008DBFC6E3E0E14E2E81E08EBFD1E0F1E06E
:100030005F2EEEEFF0E0A0E6B0E0A89584B7082EC2
:10004000877F84BF88E1992781BD91BD88278D93E3
:100050003197E9F7662480E387BB87E088BBB39BD1
:1000600001C028D280E080936900A1E6B0E0E0D230
:1000700080E08093650088E387BB87E088BB8AE0E7
:1000800090E0C5D281E080936000A6E3B0E00C91DF
:1000900001FB81E00EF480E08F93A6E3B0E00C91C9
:1000A00002FB81E00EF480E09F918923882309F40C
:1000B00001C01FD182E080936000A6E3B0E00C9104
:1000C00000FB81E00EF480E08F93A6E3B0E00C919A
:1000D00001FB81E00EF480E09F918923882309F4DD
:1000E00001C007D183E080936000A6E3B0E00C91EB
:1000F00000FB81E00EF480E08F93A6E3B0E00C916A
:1001000002FB81E00EF480E09F918923882309F4AB
:1001100001C0EFD089E287BB86E188BB8AE090E02E
:1001200076D284E080936000A6E3B0E00C9101FBFE
:1001300081E00EF480E08F93A6E3B0E00C9102FB27
:1001400081E00EF480E09F918923882309F401C0A7
:10015000D0D085E080936000A6E3B0E00C9101FB75
:1001600081E00EF480E08F93A6E3B0E00C9102FBF7
:1001700081E00EF080E09F918923882309F401C07B
:10018000B8D086E080936000A6E3B0E00C9101FB5C
:1001900081E00EF080E08F93A6E3B0E00C9102FBCB
:1001A00081E00EF480E09F918923882309F401C047
:1001B000A0D08AE287BB85E188BB8AE090E027D2A5
:1001C00087E080936000A6E3B0E00C9100FB81E043
:1001D0000EF080E08F93A6E3B0E00C9102FB81E08B
:1001E0000EF480E09F918923882309F401C081D017
:1001F00088E080936000A6E3B0E00C9100FB81E012
:100200000EF480E08F93A6E3B0E00C9102FB81E056
:100210000EF080E09F918923882309F401C069D002
:1002200089E080936000A6E3B0E00C9100FB81E0E0
:100230000EF480E08F93A6E3B0E00C9102FB81E026
:100240000EF480E09F918923882309F401C051D0E6
:100250008CE287BB83E188BB8AE090E0D8D18BE059
:1002600080936000A6E3B0E00C9100FB81E00EF00B
:1002700080E08F93A6E3B0E00C9101FB81E00EF4E7
:1002800080E09F918923882309F401C032D08AE05D
:1002900080936000A6E3B0E00C9100FB81E00EF4D7
:1002A00080E08F93A6E3B0E00C9101FB81E00EF4B7
:1002B00080E09F918923882309F401C01AD08CE043
:1002C00080936000A6E3B0E00C9100FB81E00EF4A7
:1002D00080E08F93A6E3B0E00C9101FB81E00EF08B
:1002E00080E09F918923882309F401C002D0C3CE06
:1002F000B9CEC39A84E690E08AD1C39884E690E0B0
:1003000086D100916900013009F001C02BC0009135
:100310006900023009F001C048C0009160000B3054
:1003200009F009C0A9E6B0E08C918F5F8C9380E062
:1003300080936500A0CE009160000C3009F011C0E0
:10034000EAE0F0E0A4E1B0E094E09BD1A1E6B0E007
:100350000D911D912D913C9176D109F001C09AC06B
:1003600065C032C0009160000C3009F01DC0EAE0A9
:10037000F0E0A4E1B0E094E084D1A1E6B0E00D911A
:100380001D912D913C915FD109F401C04FC058D00F
:10039000A1E6B0E04DD180E080936500A9E6B0E031
:1003A0008C918F5F8C9367CE0FC0009160000C30F2
:1003B00009F009C0EAE0F0E0A1E6B0E094E07BE7F4
:1003C0004FD13ED04FCE00C0A5E6B0E08C918F5FFC
:1003D0008C9300916500043010F009F001C001C059
:1003E00025C0A1E6B0E00D911D912D913C914AE010
:1003F00050E060E070E0BCD0A1E6B0E00D931D934A
:100400002D933D93A1E6B0E00D911D912D913C916E
:10041000A0E6B0E04C915527662777270FD1A1E6DB
:10042000B0E00D931D932D933D930895C39AE3E09F
:10043000F0E098D0C398E4E1F0E094D001D012CE7F
:1004400082E08093670088EC8093680001D0089573
:1004500084E690E0DCD081E0809366004091670004
:1004600000916600041710F009F013C0C39AA8E6C3
:10047000B0E08C919927CBD0C398A8E6B0E08C91DE
:100480009927C5D0A6E6B0E08C918F5F8C9308F4D5
:10049000E5CF0895A1E6B0E0CBD0D2DF84EF91E0C4
:1004A000B6D0C59AE2E0F0E05DD0C598E1E0F0E0BA
:1004B00059D0D8CD84E690E0AAD081E08093660040
:1004C00000916600083C10F009F00DC089E190E051
:1004D0009ED0B39901C045C0A6E6B0E08C918F5F75
:1004E0008C9308F4EDCF8FEF8093680081E08093C8
:1004F000660000916600023310F009F010C0A6E615
:10050000B0E0EC91FF27A8E6B0E091E07BE7A8D04F
:10051000A6E6B0E08C918F5F8C9308F4EACFEAE016
:10052000F0E002ED14E020E030E0A0E1BB2794E031
:100530007BE796D0B39B01C0FDCFBB9AE1E0F0E032
:1005400011D0C39A88EC90E062D0C39888EC90E018
:100550005ED0C39A88EC90E05AD0C39888EC90E0C3
:1005600056D0089588EE93E052D03197D9F7089588
:1005700022D006D000FC01D0089528D030D00895B4
:10058000842F952FA62FB72F442755276627772727
:10059000F1E2889409C020F4480F591F6A1F7B1F9D
:1005A00076956795579547953795279517950795AC
:1005B000FA9589F708950024E89477FF02C006D0E1
:1005C000689400F809D010F80124089512D04F5F04
:1005D0005F4F6F4F7F4F0895E89437FF0895009560
:1005E0001095209530950F5F1F4F2F4F3F4F689408
:1005F0000895409550956095709508953197F1F75D
:100600000895689462F80895E89462F80895EF9365
:10061000FF93EE27E82BE92B31F0EAEFF0E031977A
:10062000F1F70197D1F7FF91EF91089582E001C0B2
:1006300084E099279D938A95E9F70895040F151F83
:10064000261F371F08950417150726073707089533
:10065000E199FECFEEBB3196089591E001C092E0A2
:100660007B3751F47FB7F894F3DF8D918DBBE29A1D
:10067000E19A9A95C9F77FBF7727089591E001C065
:1006800092E0E6DFE09A8DB38D939A95D1F70895C5
:00000001FF
